:100000000C9438000C9466000C94ED000C94530092
:100010000C9453000C9453000C9453000C94530014
:100020000C9453000C9453000C9453000C94530004
:100030000C9453000C9453000C9453000C945500F2
:100040000C9453000C9453000C9453000C945300E4
:100050000C9453000C9453000C9453000C945300D4
:100060000C9453000C9453000C9453000C945300C4
:1000700011241FBECFEFD0E1DEBFCDBF12E0A0E064
:10008000B1E0E4E1FFE002C005900D92A038B107B5
:10009000D9F71FE0A0E8B2E001C01D92AE36B1076B
:1000A000E1F70C94FB030C9400001F920F920FB623
:1000B0000F9211248F93809180028F5F8093800232
:1000C0008F910F900FBE0F901F9018951F920F9257
:1000D0000FB60F9211248F939F93EF93FF93E091AC
:1000E0008102FF278091840090918500EE0FFF1F11
:1000F000E257FD4F91838083E0918102FF27809139
:100100008002E254FD4F8083E0918102FF27EA5292
:10011000F14F81E08083E0918102FF2780912901E6
:10012000F695FE2FEE27F795E795EA52FD4F858766
:10013000E0918102FF2780912A01F695FE2FEE279C
:10014000F795E795EA52FD4F8687E0918102FF27F8
:1001500080912B01F695FE2FEE27F795E795EA5251
:10016000FD4F8787E0918102FF2780912C01F69552
:10017000FE2FEE27F795E795EA52FD4F808BE09131
:100180008102FF2780912D01F695FE2FEE27F7952E
:10019000E795EA52FD4F818BE0918102FF27809124
:1001A0002E01F695FE2FEE27F795E795EA52FD4FC3
:1001B000828B809181028F5F809381028091810286
:1001C000883111F410928102FF91EF919F918F91EC
:1001D0000F900FBE0F901F9018951F920F920FB6A1
:1001E0000F9211242F933F934F935F936F937F93BD
:1001F0008F939F93AF93BF93EF93FF931DBA87E7BE
:1002000088B988B98FEF88B986B18171E9F3E09137
:100210008102FF278091840090918500EE0FFF1FDF
:10022000E257FD4F91838083E0918102FF27809107
:100230008002E254FD4F808386B18171E9F789E93C
:1002400088B988B988B988B940B193B18FEF88B9B6
:1002500020E030E077E76FEF59E9EEEEFEE078B9A5
:1002600078B968B986B18171E9F3408391832E5FD3
:100270003F4F329686B18171E9F758B958B958B9EC
:1002800058B940B193B168B92E3F310541F7409359
:10029000EC0F9093ED0F80918D02833009F490C0A4
:1002A00080918D028823A9F59091EE0E97FDC6C02E
:1002B0008091EF0E87FDE1C0981708F0A2C040E0E2
:1002C00050E0AEEEBEE0E0918102FF27CA019695B4
:1002D00087952C911296F695FE2FEE27F795E795C8
:1002E000EA52FD4FE80FF91F20834E5F5F4F81E018
:1002F0004030580741F7E0918102FF27F695FE2F25
:10030000EE27F795E795EB5AFC4F80818E7F80832F
:100310002EC080918D02813009F492C041E050E0FE
:10032000AFEEBEE0E0918102FF27CA019695879566
:100330002C911296F695FE2FEE27F795E795EA5247
:10034000FD4FE80FF91F20834E5F5F4F81E0413082
:10035000580741F7E0918102FF27F695FE2FEE271F
:10036000F795E795EB5AFC4F808181608083E0919F
:100370008102FF27EA52F14F32E03083209181025F
:10038000809181028F5F8093810280918102883108
:10039000A9F19091810280918202981751F1809188
:1003A00083028F5F8093830280918302803120F4E7
:1003B0003CBB83E08DBB63C03CBB81E08DBB5FC0B9
:1003C00020E030E0AEEEBEE0E0918102FF278D91AB
:1003D000F695FE2FEE27F795E795EA52FD4FE20FCF
:1003E000F31F80832F5F3F4F81E02030380761F794
:1003F000BECF822F992780938102D1CF10928102A4
:10040000C8CF41E050E0AFEEBEE0E0918102FF27AF
:10041000CA01969587952C911296F695FE2FEE2798
:10042000F795E795EA52FD4FE80FF91F20834E5FDD
:100430005F4F81E04130580741F78CCF909538CF1E
:1004400040E050E0AEEEBEE0E0918102FF27CA013D
:10045000969587952C911296F695FE2FEE27F79597
:10046000E795EA52FD4FE80FF91F20834E5F5F4F7B
:1004700081E04030580741F73ECF80951DCFFF9176
:10048000EF91BF91AF919F918F917F916F915F910C
:100490004F913F912F910F900FBE0F901F90189585
:1004A0008F708A3018F0895C99270895805D9927AC
:1004B000089560E070E080917F028F7E80937F02DC
:1004C00020E030E040E050E080917F028BB92F5F68
:1004D0003F4F4F4F5F4F203888E3380781E0480790
:1004E00080E0580789F780917F02806180937F02C6
:1004F00020E030E040E050E080917F028BB92F5F38
:100500003F4F4F4F5F4F203888E3380781E048075F
:1005100080E0580789F780917F028F7D80937F026A
:1005200020E030E040E050E080917F028BB92F5F07
:100530003F4F4F4F5F4F203888E3380781E048072F
:1005400080E0580789F780917F02806280937F0264
:1005500020E030E040E050E080917F028BB92F5FD7
:100560003F4F4F4F5F4F203888E3380781E04807FF
:1005700080E0580789F780917F028F7B80937F020C
:1005800020E030E040E050E080917F028BB92F5FA7
:100590003F4F4F4F5F4F203888E3380781E04807CF
:1005A00080E0580789F780917F02806480937F0202
:1005B00020E030E040E050E080917F028BB92F5F77
:1005C0003F4F4F4F5F4F203888E3380781E048079F
:1005D00080E0580789F76F5F7F4F6430710509F03D
:1005E0006ACF0895982F80918502873028F5292FAA
:1005F000332780918502E0917302F0917402E80F35
:10060000F11D8081992787FD90952817390709F4F6
:1006100046C041E080918502E0917D02F0917E022A
:10062000E80FF11D8081992787FD909528173907DC
:1006300009F44BC0442341F5809185028F5F80937C
:10064000850280918502873080F01092850280912A
:100650008902873058F480918A02873038F51092E9
:100660008A0280918A0280938902089510928A02F8
:1006700080918A0280938902809184028F5F8093A7
:10068000840210928802089510928502809185025A
:1006900080938A0280918A028093890208958091D2
:1006A00089028F5F8093890240E0B4CF10928A0262
:1006B00080918A0280938902809184028F5F809367
:1006C000840281E080938802089580918A028F5F7E
:1006D00080938A02B1CF982F8C32A1F0809185024D
:1006E000841778F480918502262F280F312D311D33
:1006F000F901E45EFE4F9083809185028F5F8093C5
:1007000085020895809184028F5F80938402109205
:1007100085020895982F8C32F1F08091850284171C
:10072000C8F4903309F452C080918502462F480FD7
:10073000512D511DFA01E45EFE4F908381E08093BC
:100740008C029E3209F454C0809185028F5F8093A1
:10075000850208950895809184028F5F80938402BA
:1007600080918502841758F580918B02882381F44B
:1007700080918502262F280F312D311DF901E45E6D
:10078000FE4F8EE28083809185028F5F8093850289
:1007900080918502841798F4772790E380918502F1
:1007A000FB01E80FF11DE45EFE4F9083809185020E
:1007B0008F5F8093850280918502841778F3109271
:1007C000850210928B0210928C02089520918C0267
:1007D000213009F0B9CF80918502462F480F512D65
:1007E000511DFA01E45EFE4F908320938C02ACCF42
:1007F00080938B02A9CFCFEFD0E1DEBFCDBF11B880
:100800009FEF92B914B895B98EEE87B998B980E781
:100810008AB98FE88BB982E08093810081E0809370
:100820006F0015BE8BE08093690083E08DBB7894E8
:1008300010928D0289B18078803809F469C310E084
:1008400080918D02833019F08DE4809360010E94C5
:100850005902103409F459C3103809F453C3112351
:1008600009F04DC390E08FE19093C5008093C400E0
:1008700088E18093C10086E08093C200A0911A01B4
:10088000B0911B018C91882369F0FD013196809114
:10089000C00085FFFCCF8C918093C600DF01819161
:1008A0008823A9F7FF248091C00087FD56C090914E
:1008B0008102809182029817B1F3E0918202FF27B2
:1008C000EA52F14F8081813009F467C0E0918202E1
:1008D000FF27EA52F14F8081823029F7809186020A
:1008E00090918702892B09F47DC1809186029091B5
:1008F0008702019709F437C280918602909187029E
:10090000029708F4D9C180918602909187028E5097
:10091000914008F0D1C18091C00085FFC4CFE09123
:100920008602F0918702E45AFE4F80818093C600D0
:10093000E0918602F0918702E45AFE4F8081F8260A
:10094000809186029091870201969093870280930E
:1009500086028091C00087FFAACF9091C600809147
:100960008402882309F4D0C080918802882309F08A
:10097000B6C080918402853009F447C2863008F001
:1009800033C2823009F484C2833008F063C28130FC
:1009900009F4A9C2109284028ACF809186029091B4
:1009A0008702892B09F4B4C0809186029091870256
:1009B000892BD1F080918602909187020E97A0F446
:1009C0008091C00085FF6FCFE0918602F091870291
:1009D000E55EFE4F80818093C600E0918602F09133
:1009E0008702E55EFE4FAACF809186029091870232
:1009F0000E9770F18091860290918702449740F59E
:100A00008091C00085FF4FCF809182029927E091AD
:100A10008602F09187029695982F8827979587955B
:100A2000E80FF91FEB52FD4F80818093C600809143
:100A300082029927E0918602F09187029695982F7D
:100A4000882797958795E80FF91FEB52FD4F76CFD2
:100A50008091860290918702449740F080918602AF
:100A6000909187028234910508F4AACF8091860282
:100A7000909187028234910509F460C180918602C9
:100A8000909187028334910509F4C5C18091860253
:100A9000909187028434910509F4C3C18091860244
:100AA000909187028534910509F4CCC180917F0231
:100AB000806480937F0280917F028BB910928702BD
:100AC00010928602809182028F5F809382028091D1
:100AD0008202883109F401C283E08DBBE4CE8091AB
:100AE0008402853059F0863008F06CC1823031F0D4
:100AF000833008F0C1C1813009F04CCF40E060E0A4
:100B0000892F0E946B03D3CE892F0E94F202CFCE91
:100B100080917F028F7B80937F0280917F028BB9CF
:100B2000E0918202FF27E254FD4F808182958F7011
:100B30000E94500280932001E0918202FF27E2543C
:100B4000FD4F80810E94500280932101E09182023A
:100B5000FF27EE0FFF1FE257FD4F80819181892F04
:100B6000992782958F700E94500280932201E09114
:100B70008202FF27EE0FFF1FE257FD4F8081918118
:100B8000892F99270E94500280932301E0918202CD
:100B9000FF27EE0FFF1FE257FD4F80819181929555
:100BA00082958F7089279F7089270E9450028093B9
:100BB0002401E0918202FF27EE0FFF1FE257FD4F55
:100BC000808191810E94500280932501809186024C
:100BD00090918702019690938702809386020EE09F
:100BE000F02E61CE80917F028F7E80937F02809174
:100BF0007F028BB9E0918202FF27E254FD4F808192
:100C000082958F700E94500280936201E09182026F
:100C1000FF27E254FD4F80810E94500280936301C0
:100C2000E0918202FF27EE0FFF1FE257FD4F808108
:100C30009181892F992782958F700E94500280930D
:100C40006401E0918202FF27EE0FFF1FE257FD4F84
:100C500080819181892F99270E945002809365019C
:100C6000E0918202FF27EE0FFF1FE257FD4F8081C8
:100C70009181929582958F7089279F7089270E9414
:100C8000500280936601E0918202FF27EE0FFF1F62
:100C9000E257FD4F808191810E945002809367014D
:100CA00080918602909187020196909387028093AB
:100CB00086029EE0F92EF7CD809186029091870200
:100CC0008E509140D9F180918602909187028F5089
:100CD000914009F4A0C080918602909187028051D2
:100CE000914009F49EC080918602909187028151C3
:100CF000914009F4A7C080917F02806180937F02B8
:100D000080917F028BB910928702109286028091A7
:100D100082028F5F8093820280918202883109F47F
:100D2000DFC080918302815080938302809183028F
:100D3000803108F0B8CD82E08CBBCECE8091C0006F
:100D400085FFB1CD8F2D82958F700E9450028093C8
:100D5000C600809186029091870201969093870247
:100D600080938602A0CDC0E0D0E009E611E0E091DA
:100D70008202FF27F695FE2FEE27F795E795EA52B8
:100D8000FD4FEC0FFD1F808182958F700E945002F5
:100D9000F8018083E0918202FF27F695FE2FEE276F
:100DA000F795E795EA52FD4FEC0FFD1F80812196E4
:100DB0000E945002F80181830E5F1F4FC038D10599
:100DC000B1F6BECD873009F479C0873008F496CEED
:100DD000883009F493CE893009F0DCCD45E064E336
:100DE000892F0E948A0363CD873009F487CE87302C
:100DF000E8F1883009F482CE893009F0CBCD46E0A5
:100E000064E1892F0E946B0352CD4AE067E2892F8B
:100E10000E946B034CCD8091C00085FF44CD8F2D87
:100E200094CF8091C00085FF3ECD8DE08093C600B9
:100E30008091860290918702019690938702809319
:100E4000860231CD8091C00085FF2DCD8AE0809350
:100E5000C60076CD833009F44CC0843009F09ACDB9
:100E600041E065E2892F0E946B0321CD41E062E3FE
:100E7000892F0E946B031BCD833009F43FCE843051
:100E800009F088CD40E060E0892F0E946B030FCD10
:100E900041E06BE0892F0E946B0380912701813430
:100EA00099F080912E0180FD0FC080917F028062B9
:100EB00080937F0280917F028BB9F9CC42E06AE394
:100EC000892F0E946B03F3CC80917F028F7D8093EA
:100ED0007F0280917F028BB9EACC10928202FCCD16
:100EE000109282021ECF46E06DE0892F0E946B03B4
:100EF000DECC49E06BE1892F0E946B03D8CC91E0F6
:100F000083E0B2CC90E080E4AFCC90E081E8ACCC60
:040F100010EC96CC7F
:100F14000D0A4669726D7761726520566572736950
:100F24006F6E3A203237630D0A0000012442532CBD
:100F34003030303030302C2D2C3030303030302CBC
:100F44003030303030302C303030302E30303030A3
:100F54002C2D2C30303030302E303030302C2D2CA5
:100F640030303030302C30302C3237622A0024427A
:100F7400442C3030303030302C3030303030303061
:100F8400303030303030303030303030303030305D
:100F9400303030303030303030303030303030304D
:100FA400303030303030303030303030303030303D
:100FB400303030303030303030303030303030302D
:100FC400303030303030303030303030303030301D
:100FD400303030303030303030303030303030300D
:100FE40030303030303030303030303030303030FD
:100FF40030303030303030303030303030303030ED
:1010040030303030303030303030303030303030DC
:1010140030303030303030303030303030303030CC
:1010240030303030303030303030303030303030BC
:1010340030303030303030303030303030303030AC
:10104400303030303030303030303030303030309C
:10105400303030303030303030303030303030308C
:10106400303030303030303030303030303030307C
:101074003030303030303030302A00244750524D38
:10108400432C006B022447504747412C007502FF54
:00000001FF
